:100000000C94D1040C9419050C9419050C94190541
:100010000C9419050C9419050C9419050C941905E8
:100020000C9419050C9419050C9419050C94A81C32
:100030000C9419050C947F1C0C9419050C9419054B
:100040000C9419050C9419050C9419050C94591C61
:100050000C9419050C9419050C9419050C941905A8
:100060000C9419050C9419050C9419050C94190598
:100070000C9419050631FF0974A1010975150026B4
:10008000FF009520750881020976150026FF00956E
:100090002075089102C005010902A1010901A10012
:1000A0008501050919012908150025019508750123
:1000B00081020501093009311581257F95027508F6
:1000C000810609381581257F950175088106050C83
:1000D0000A38021581257F950175088106C0C00583
:1000E000010980A10185021601002637001A81004E
:1000F0002AB700751095018100C0050C0901A10106
:100100008503160100269C021A01002A9C02751024
:1001100095018100C005010906A101050719E02923
:10012000E715002501950875018102950175088183
:1001300001050819012905950575019102950175BB
:100140000391010507190029FF150026FF009506F8
:1001500075088100C02530325820002530325820E3
:10016000005B204E655854206B6579626F61726444
:1001700020696E697469616C697A6564205D0A0042
:100180005B20496E7469616C697A696E67204E659F
:100190005854206B6579626F617264205D0A002596
:1001A000583A2530386225730A000A20203031324F
:1001B00033343536370A004C45443A20253032581E
:1001C0000A000A4C6F6F702073746172742E0A00FB
:1001D0000A55534220636F6E666967757265642EB7
:1001E0000A000A544D4B3A6333626438342F4C553D
:1001F00046413A6436613764660A005B535D005BD2
:10020000575D005B525D005B695D005B49256420C2
:10021000253034585D005B50256420253034585D0E
:10022000005B705D005B4C256420253032585D001A
:100230005B7225645D0009025400030100A03209CD
:100240000400000103010100092111010001224005
:10025000000705810308000A0904010001030102E7
:1002600000092111010001227F0007058203080017
:10027000010904020001030000000921110100012D
:100280002222000705830320000112011001000053
:100290000008EDFEBCBC0005010200013E034E005B
:1002A00065005800540020004B0065007900620092
:1002B0006F00610072006400200074006F00200075
:1002C000550053004200200063006F006E0076006E
:1002D0006500720074006500720000000E03740077
:1002E0002E006D002E006B002E0000000403090498
:1002F0005B635D0073797374656D3A202530345803
:100300000A00636F6E73756D65723A20253034583C
:100310000A003F004D3E2000433E20000A002575A4
:1003200000363A20776865656C5F74696D655F7447
:100330006F5F6D61783A20000A00257500353A201C
:10034000776865656C5F6D61785F73706565643A49
:1003500020000A00257500343A2074696D655F74C9
:100360006F5F6D61783A20000A00257500333A20EE
:100370006D61785F73706565643A20000A002575C9
:1003800000323A20696E74657276616C286D73294B
:100390003A20000A00257500313A2064656C6179C5
:1003A000282A31306D73293A20000A092D20566120
:1003B0006C756573202D0A004D3E004D25643E206E
:1003C000003F007365742064656661756C740A0093
:1003D000433E20000A002530325820006B657962C8
:1003E0006F6172643A2000804E4C31302F0C121332
:1003F000508062635880514F595C5E5B66525A5D13
:100400004B492A2E2D2526275F6061575653545598
:10041000802834330F3637381D1B06190510112C70
:10042000041607090A0E0D0B2B141A0815181C17B1
:10043000351E1F20212423227C78657B7D79394A53
:1004400080808080808080290A002575002F00250B
:1004500075005D280025640020002564002000252B
:10046000640020002564007C0025303258006D6F48
:100470007573656B6579205B62746E7C782079207A
:100480007620685D287265702F61636C293A205B65
:10049000000A092D204D61676963202D0A643A091D
:1004A00064656275670A783A096465627567206DEC
:1004B00061747269780A6B3A096465627567206BCA
:1004C0006579626F6172640A6D3A09646562756785
:1004D000206D6F7573650A763A0976657273696F78
:1004E0006E0A733A097374617475730A633A096327
:1004F0006F6E736F6C65206D6F64650A302D343AD2
:10050000096C61796572302D34284631302D4634BE
:10051000290A506175733A09626F6F746C6F616478
:1005200065720A000A092D20436F6E736F6C652097
:100530002D0A4553432F713A09717569740A6D3A52
:10054000096D6F7573656B65790A003F0074696D9D
:1005500065725F72656164333228293A2025303430
:100560006C580A006B6579626F6172645F69646CD4
:10057000653A2025580A006B6579626F6172645F85
:1005800070726F746F636F6C3A2025580A00686F41
:1005900073745F6B6579626F6172645F6C656473BD
:1005A00028293A2025580A000A092D20537461741D
:1005B0007573202D0A004743433A20372E332E30DF
:1005C000204156522D4C4942433A20322E302E3093
:1005D000204156525F415243483A2061767233358A
:1005E0000A004F5054494F4E533A204C5546412033
:1005F0004D4F5553454B45592045585452414B4555
:100600005920434F4E534F4C4520434F4D4D414E83
:1006100044204B45594D41505F53454354494F4E3B
:1006200020343039360A004255494C443A2063336D
:1006300062643834202831333A32323A313320463A
:1006400065622032372032303233290A005649445D
:100650003A2030784645454428742E6D2E6B2E295D
:10066000205049443A20307842434243284E65584E
:1006700054204B6579626F61726420746F2055530A
:100680004220636F6E7665727465722920564552FA
:100690003A203078303530300A00444553433A2010
:1006A00055534220636F6E76657274657220666F73
:1006B00072204E655854206E6F6E2D414442204B7F
:1006C0006579626F6172640A000A092D20566572AD
:1006D00073696F6E202D0A000A6D6F7573653A207D
:1006E0006F66660A000A6D6F7573653A206F6E0A51
:1006F000000A6B6579626F6172643A206F66660A00
:10070000000A6B6579626F6172643A206F6E0A004D
:100710000A6D61747269783A206F66660A000A6D24
:1007200061747269783A206F6E0A000A64656275B6
:10073000673A206F6E0A000A64656275673A206F37
:1007400066660A000A0A626F6F746C6F6164657294
:100750002E2E2E2000433E20006D6B5F776865656E
:100760006C5F74696D655F746F5F6D6178203D20AB
:1007700025640A006D6B5F776865656C5F6D6178F5
:100780005F7370656564203D2025640A006D6B5FB2
:1007900074696D655F746F5F6D6178203D202564BD
:1007A0000A006D6B5F6D61785F7370656564203DF5
:1007B0002025640A006D6B5F696E74657276616CEA
:1007C000203D2025640A006D6B5F64656C617920B3
:1007D0003D2025640A006D6B5F776865656C5F740A
:1007E000696D655F746F5F6D6178203D2025640AD7
:1007F000006D6B5F776865656C5F6D61785F7370C6
:10080000656564203D2025640A006D6B5F74696D29
:10081000655F746F5F6D6178203D2025640A006D0F
:100820006B5F6D61785F7370656564203D20256442
:100830000A006D6B5F696E74657276616C203D2095
:1008400025640A006D6B5F64656C6179203D20252D
:10085000640A0077686572652064656C74613A208B
:10086000637572736F723D25642C20776865656CC3
:100870003D25640A53656520687474703A2F2F65AE
:100880006E2E77696B6970656469612E6F72672F70
:1008900077696B692F4D6F7573655F6B6579730A47
:1008A000000A092D204D6F7573656B6579202D0A3F
:1008B0004553432F713A09717569740A313A0964D5
:1008C000656C6179282A31306D73290A323A0969D9
:1008D0006E74657276616C286D73290A333A096DFE
:1008E00061785F73706565640A343A0974696D658F
:1008F0005F746F5F6D61780A353A09776865656C7A
:100900005F6D61785F73706565640A363A09776870
:1009100065656C5F74696D655F746F5F6D61780AA2
:100920000A703A097072696E742076616C7565732D
:100930000A643A097365742064656661756C747342
:100940000A75703A092B310A646F776E3A092D31B6
:100950000A706775703A092B31300A7067646F77D7
:100960006E3A092D31300A0A7370656564203D20A6
:1009700064656C7461202A206D61785F73706565B1
:1009800064202A2028726570656174202F207469A4
:100990006D655F746F5F6D6178290A004C25640A8C
:1009A000000011241FBECFEFD4E0DEBFCDBF04B6E0
:1009B00003FE28C080912A0390912B03A0912C0361
:1009C000B0912D038730904BA740B04BD9F41092D3
:1009D0002A0310922B0310922C0310922D0314BEA5
:1009E0000FB6F894A89580916000886180936000AC
:1009F000109260000FBE1092010810920008E0E013
:100A0000F8E3099511E0A0E0B1E0E4E8F4E402C005
:100A100005900D92A233B107D9F723E0A2E3B1E02C
:100A200001C01D92AA32B207E1F70E94651D0C9425
:100A300040220C940000FF93EF93E0913201F0917B
:100A40003301309709F00995EF91FF910895FC016A
:100A50008591803011F0EFDFFBCF0895FF27E0E2B2
:100A600030E247FF0CC0419597FF09C0EDE2609569
:100A7000709580959095611D711D811D911D27FFB9
:100A800002C0219530E350E2AA27660F771F881F26
:100A9000991FAA1FA41710F0A41B63955A95A9F7D4
:100AA000AA3008F0A95FA05DAF93F39561157105B9
:100AB0008105910541F7ED3211F4EF93F395F217AB
:100AC00018F43F93F395FBCF8F91B5DFFA95E1F7DB
:100AD0000895E991F9918591803021F0853219F0DE
:100AE000AADFF9CF089520E0E89455915532C1F37B
:100AF000503311F4689455915A3348F4505390F39D
:100B0000220F022E220F220F200D250FF4CF0EF4FC
:100B1000219589919991533619F3533729F153351A
:100B200059F1BC0188279927E8945C3621F4899112
:100B3000999168945591543639F446EF7EF077FFD9
:100B40000DC08FEF9FEF0AC055374AE039F0583596
:100B500040E121F0523642E009F00895FF93EF930F
:100B60007DDFEF91FF91B7CFFF93EF93FC01819170
:100B70008030B9F360DFFBCFFF93EF9368DFF1CFF5
:100B8000DF93CF93CDB7DEB72596A3DFCF91DF916B
:100B900008958091140380FF0CC06091130170E0F0
:100BA00075956795759567956115710559F1862F4E
:100BB000089581FF06C06091130170E075956795F7
:100BC000F3CF6091130170E082FD0CC060911503BA
:100BD0006623A9F0209112018091130190E0621721
:100BE00030F0BC0160387105F8F28FE7089570E0CD
:100BF0000E940122622F70E00E941222F3CF61E076
:100C000070E0D5CF81E008958091140380FF11C07A
:100C10008091150190E065E070E00E9401229595B9
:100C200087959595879580389105B0F50097B1F136
:100C3000089581FF0AC08091150190E065E070E0A1
:100C40000E94012295958795EECF82FF08C0809182
:100C5000150190E065E070E00E940122E4CF309140
:100C600015033323B1F0209114018091150190E018
:100C700065E070E00E940122BC013217A0F6832FCC
:100C800090E00E940122622F70E00E941222CB01AC
:100C9000CACF85E090E008958FE7089581E0089538
:100CA000E72FF0E093E0EE0FFF1F9A95E1F7E60FD4
:100CB000F11DE951FC4F6491E62FE295E77090E059
:100CC00023E0880F991F2A95E1F78E0F911D34E0DC
:100CD000880F991F3A95E1F7E62FEF70E80FF92F8B
:100CE000F11DEE0FFF1FE050F84985919491089592
:100CF0002FB7F89480911F0390912003A0912103B6
:100D0000B09122032FBF08954F925F926F927F920E
:100D10009F92AF92BF92CF92DF92EF92FF920F938A
:100D20001F93CF93DF9300D000D01F92CDB7DEB7D3
:100D30006B837C838D837A018C819D81892B49F023
:100D40008FEFF81204C081E09FEF491719F080E09F
:100D500001C081E080FD6AC00F2D10E0CE2CD12CA7
:100D60008B81882309F456C04090AC025090AD02AC
:100D70006090AE027090AF0280912603909127039D
:100D8000A0912803B0912903482A592A6A2A7B2A6C
:100D90002FE1A22EB12C9A2CD301C2010A2C04C03F
:100DA000B695A795979587950A94D2F780FD2BC0A5
:100DB00081E0A81AB10878F7912CF80193E0EE0FC2
:100DC000FF1F9A95E1F7E055FD4FEC0DFD1D908258
:100DD000E982FA8269817A81892D0F900F900F90B4
:100DE0000F900F90DF91CF911F910F91FF90EF9097
:100DF000DF90CF90BF90AF909F907F906F905F906B
:100E00004F900C945006B7018A2D0E94500601970E
:100E100079F2D3CFF80183E0EE0FFF1F8A95E1F757
:100E2000E055FD4FEC0DFD1D9080D2CF90E080E0AD
:100E30000F900F900F900F900F90DF91CF911F9117
:100E40000F91FF90EF90DF90CF90BF90AF909F9069
:100E50007F906F905F904F90089541E050E060E088
:100E600070E004C0440F551F661F771F8A95D2F7A4
:100E700040955095609570958091AC029091AD022F
:100E8000A091AE02B091AF0284239523A623B7238D
:100E90008093AC029093AD02A093AE02B093AF02E8
:100EA000089541E050E060E070E004C0440F551F39
:100EB000661F771F8A95D2F78091AC029091AD02A0
:100EC000A091AE02B091AF02842B952BA62BB72B2D
:100ED0008093AC029093AD02A093AE02B093AF02A8
:100EE00008958091AB0290917A02981301C0089501
:100EF0008F5F8770FACF1F93CF93DF9300D000D01E
:100F00001F92CDB7DEB7942F4983252F5A836B8369
:100F10007C838D834C815D8181E0452B31F02F3FB7
:100F200019F481E09F3F09F080E0182F117080FDD7
:100F30002CC049815A816B817C818D810E948406FD
:100F4000292F22952F702C3078F42A30A8F42250C3
:100F50002230C8F0812F0F900F900F900F900F90BC
:100F6000DF91CF911F9108952C3011F02F3091F720
:100F700093FB112710F9EECF803C28F0803E50F310
:100F8000815F833038F311E0E5CF10E0E3CFE091EB
:100F90001603F0911703309721F00190F081E02DB6
:100FA000099480E008951092E2001092E100E0EED2
:100FB000F0E0808181608083E8EDF0E080818F77D0
:100FC000808319BCE3E6F0E0808181608083109229
:100FD000580208950E94D307F89487E797E7909303
:100FE00001088093000887E090EBDC0180932A03DE
:100FF00090932B03A0932C03B0932D0388E19CE0E6
:101000000FB6F894A895809360000FBE909360008F
:10101000FFCFFC0180916C0290916D0286179707BB
:10102000A0F06115710529F49091E8009E779093E6
:10103000E80090E06115710551F4911108C08091AC
:10104000E80082FF32C080E00895BC01F2CF8091B9
:101050006E028823B1F18530B1F18091E80083FD03
:101060002EC08091E80082FDEACF8091E80080FFE9
:10107000E1CF2091F20030E06115710519F02830C0
:10108000310558F091E02830310509F090E02091C9
:10109000E8002E772093E800CDCF81918093F10076
:1010A000615071092F5F3F4FE7CF80916E02882317
:1010B00041F0853041F08091E80083FFC0CF81E0AE
:1010C000089582E0089583E008952091E40030912E
:1010D000E50085E69091EC0090FF06C09091E80055
:1010E00090FF06C080E008959091E80092FDFACF4D
:1010F00090916E02992391F0953091F09091EB00D0
:1011000095FD10C04091E4005091E500241735078B
:1011100009F381509A01F1F684E0089582E0089580
:1011200083E0089581E008958091660287FF13C0EF
:101130008091E80082FF06C08091E8008B77809361
:10114000E80004C080916E028111F2CF0895809171
:101150006E028823D9F38091E80080FFF8CF809158
:10116000E8008E77ECCF982F9093E900242F762F0C
:1011700050E0891731F07091EC002091ED00509112
:10118000F00021FD07C09F5F953071F78093E90063
:1011900081E008953091EB003E7F3093EB00309179
:1011A000ED003D7F3093ED003091EB0031603093E6
:1011B000EB007093EC002093ED005093F000209131
:1011C000EE0027FDE0CF80E0089580915A02089557
:1011D00080913C02811113C09FB7F89440911F0386
:1011E0005091200360912103709122039FBF443CE2
:1011F00059406105710518F081E080933C02089523
:10120000EF92FF920F931F93CF93DF93D82F0FB6D8
:1012100007FE46C080916E02843079F08091030110
:1012200090E001962091050130E0822393232091E4
:1012300004012817190609F0C9C00E94E8088111A5
:101240000FC08091030190E001962091050130E0EC
:1012500082239323209104012817190609F0B6C0B0
:101260000E9478068C01C091E900CF708091EC005B
:1012700080FD37C080E0C82B83E08093E90085E0E3
:10128000E82E8091EB0085FD08C08091EB0080FF87
:1012900004C08091EE0087FD44C0CF70C093E90088
:1012A000E09103018E2F90E001962091050130E03E
:1012B00082239323209104012817190609F47EC084
:1012C0008091010190910201E80FF92FF11DD08367
:1012D000809103018F5F9091050189238093030121
:1012E0006DC080E8C8CFE0910101F0910201E80FE4
:1012F000F11D90818F5F209105018223809304016D
:101300009093F1008091E80085FD0BC08091E8008A
:1013100080FF07C08091E8008E778093E800E0921C
:1013200000018091040190910301981741F190917F
:10133000E80095FDD8CF80E029C01092F1002EC0C2
:101340008091030190E001962091050130E0822315
:101350009323209104012817190609F09ECFF090DD
:101360000001FF2009F499CF0E94780680179107A9
:1013700009F487CFFA94F09200018C0182CF80911A
:10138000E80085FFD8CFD093F10081E09091F20082
:10139000992379F09091E80090FF0BC09091E800BC
:1013A00095FDCBCF9091E8009E779093E800E09276
:1013B0000001882329F2CF70C093E90080E0DF911B
:1013C000CF911F910F91FF90EF900895E09103014D
:1013D00077CF5198599A08955998519A0895833022
:1013E000C9F128F4813061F0823019F10895853017
:1013F00009F452C008F43FC0863009F45EC0089575
:1014000080911701681790F4861B809317018091D3
:1014100017011F928F9384E498E09F938F930E940B
:10142000C0050F900F900F900F9008951092170124
:10143000EECF80911601681750F4861B8093160139
:10144000809116011F928F9382E398E0E6CF10926D
:101450001601F6CF80911501681750F4861B809312
:101460001501809115011F928F938FE198E0D5CFE0
:1014700010921501F6CF80911401681750F4861B65
:1014800080931401809114011F928F938AE098E059
:10149000C4CF10921401F6CF80911301681750F455
:1014A000861B80931301809113011F928F9381EF0C
:1014B00097E0B3CF10921301F6CF80911201681715
:1014C00050F4861B80931201809112011F928F931A
:1014D00086ED97E0A2CF10921201F6CF833009F487
:1014E00045C028F4813061F0823049F1089585309B
:1014F00009F46AC008F451C0863009F47CC008952C
:1015000080911701482F460F5527551F4F3F510512
:1015100094F4680F60931701809117011F928F93C5
:1015200087EC97E09F938F930E94C0050F900F90D8
:101530000F900F9008958FEF80931701EDCF80915A
:101540001601482F460F5527551F4F3F510554F49C
:10155000680F60931601809116011F928F9385EB9F
:1015600097E0E0CF8FEF80931601F5CF80911501C2
:10157000482F460F5527551F4F3F510554F4680F0C
:1015800060931501809115011F928F9382EA97E075
:10159000C9CF8FEF80931501F5CF80911401482FAB
:1015A000460F5527551F4F3F510554F4680F609360
:1015B0001401809114011F928F938DE897E0B2CFB0
:1015C0008FEF80931401F5CF80911301482F460FC0
:1015D0005527551F4F3F510554F4680F6093130171
:1015E000809113011F928F9384E797E09BCF8FEF39
:1015F00080931301F5CF80911201482F460F552794
:10160000551F4F3F510554F4680F609312018091AC
:1016100012011F928F9389E597E084CF8FEF80931B
:101620001201F5CFCF93DF932091710230917202B6
:101630002817390701F19093720280937102E091AB
:101640001603F09117033097B1F0EC010084F18597
:10165000E02D0995809125038570853061F4DF9335
:10166000CF9382E093E09F938F930E94C0050F90E9
:101670000F900F900F90DF91CF910895CF93DF934C
:1016800020916F02309170022817390701F1909371
:10169000700280936F02E0911603F0911703309768
:1016A000B1F0EC010680F781E02D099580912503CA
:1016B0008570853061F4DF93CF9384EF92E09F9340
:1016C0008F930E94C0050F900F900F900F90DF91A5
:1016D000CF910895E82FE695E695E695F0E0E35C76
:1016E000FD4F9081482F477021E030E002C0220F6B
:1016F000331F4A95E2F7492F50E042235323452BED
:10170000A1F02095292320839091250390FF0DC0FF
:1017100080681F928F938BE591E09F938F930E9437
:10172000C0050F900F900F900F900895E82FE69549
:10173000E695E695F0E0E35CFD4F9081482F477019
:1017400021E030E002C0220F331F4A95E2F7492F13
:1017500050E042235323452B91F4922B9083909198
:10176000250390FF0CC01F928F9385E591E09F9316
:101770008F930E94C0050F900F900F900F900895C7
:1017800081EA98E00E9427051F9281E08F931F92C3
:1017900085E08F9383E598E09F938F930E94C00527
:1017A0000F900F900F900F900F900F900895CF9380
:1017B0008091250383FF7EC08EE694E00E9427057A
:1017C00080911A031F928F9389E694E09F938F93E1
:1017D0000E94C00587E694E00E94270580911B03C4
:1017E000282F082E000C330B3F938F9384E694E050
:1017F0009F938F930E94C00582E694E00E94270584
:1018000080911C03282F082E000C330B3F938F93DD
:101810008FE594E09F938F930E94C0058DE594E03F
:101820000E94270580911D03282F082E000C330BE2
:101830003F938F938AE594E09F938F930E94C00516
:1018400088E594E00E94270580911E03282F082E2A
:10185000000C330B3F938F9385E594E09F938F9318
:101860000E94C00582E594E00E942705809115033F
:101870001F928F938FE494E09F938F930E94C005F3
:101880008DE494E00E942705809114031F928F93AA
:101890008AE494E09F938F930E94C00587E494E0CC
:1018A0000E9427058DB79EB74C960FB6F8949EBF41
:1018B0000FBE8DBFE0911603F0911703309751F0E2
:1018C000C0911A030480F581E02D8AE193E0099527
:1018D000C0931A030E94780690931903809318030B
:1018E000CF9108950F931F93CF93DF9380911203AD
:1018F00090911103892B80933402909110039923C6
:1019000089F0892B80933402E5E3F2E02CE332E0A6
:1019100080E0919191118F5F2E173F07D1F78111D0
:1019200010921003E0911603F09117033097B1F174
:101930000280F381E02D84E392E0099580912503F4
:1019400082FF2CC080FF04C08CED93E00E9427052D
:10195000D0E0C0E006ED13E08091250380FF0EC0CB
:10196000FE01EC5CFD4F80811F928F931F930F93BC
:101970000E94C0050F900F900F900F902196C830D5
:10198000D10551F78091250380FF08C084ED93E0D5
:10199000DF91CF911F910F910C942705DF91CF918B
:1019A0001F910F9108951092120310921103E4E316
:1019B000F2E011821282138214821582168217823B
:1019C0000E94720C85E0EAE1F3E0DF011D928A9546
:1019D000E9F710921503109214030E94D70B90E0C0
:1019E00080E00E943E0B90E080E00C94120BCF93BD
:1019F000C82F1F928F938CE999E09F938F930E9439
:101A0000C00581E090E0A0E0B0E004C0880F991F1D
:101A1000AA1FBB1FCA95D2F7809326039093270372
:101A2000A0932803B09329030F900F900F900F906D
:101A3000CF910C94D30C882341F0809590911203A0
:101A40008923809312030C94720C0895882339F033
:101A500090911203892B809312030C94720C0895B9
:101A60008823B1F19CEF980F913A70F4E4E3F2E02F
:101A70002AE332E09281891301C0128231962E1737
:101A80003F07C1F70C94720C90E2980F983088F4DD
:101A9000877021E030E0A90102C0440F551F8A95EC
:101AA000E2F7CA0180959091120389238093120373
:101AB000E9CF9BE5980F933020F490E080E00C9400
:101AC0003E0B885A873120F490E080E00C94120B92
:101AD00008950F931F93CF93DF93CDB7DEB7AA97E7
:101AE0000FB6F894DEBF0FBECDBF80916E02882383
:101AF00009F4B1C11091E9001F708091EC0080FFE2
:101B000039C080E8182B1092E9008091E80083FF2B
:101B10009FC1E6E6F2E08EE692E02091F10021938B
:101B20008E179F07D1F780916702833009F496C022
:101B300018F5813009F45DC0823009F430C180911C
:101B4000E80083FF77C180916602909167029A3026
:101B500008F070C1E92FF0E0E055F24F0C94262216
:101B6000ED0E130F1A0F130F1A0F750F970F1A0F91
:101B700092109F1080E0C6CF8A3009F4F3C08B30FA
:101B800009F4ABC08930D9F6809166028132B9F68A
:101B900080916A0290916B02892B89F68091E8000E
:101BA000877F8093E8008091E80082FF52C0809197
:101BB000F10080935A028091E8008B778093E800CF
:101BC0000E94940880915A021F928F9380916B0219
:101BD0008F9380916A028F9385E292E09F938F9317
:101BE0000E94C0050F900F900F900F900F900F90D4
:101BF000A6CF80916602813A09F0A1CF8091E800DA
:101C0000877F8093E80080916A0290916B02892B14
:101C1000E1F060E090E080E070E00E9409088091CF
:101C2000E8008B778093E80080916B028F9380911E
:101C30006A028F9380E392E09F938F930E94C00586
:101C40000F900F900F900F907ACF68E08BE592E0A5
:101C5000E3CF80916E028111A6CF71CF8091660291
:101C6000813A09F06CCF80916A0290916B02892BC6
:101C7000C1F48091E800877F8093E8008091E800BC
:101C800080FFFCCF809111018093F1008091E800EA
:101C90008E778093E8000E94940881E292E00E948F
:101CA000270580916A0290916B02019709F047CF56
:101CB0008091E800877F8093E8008091E80080FFB2
:101CC000FCCF809110018093F1008091E8008E7725
:101CD0008093E8000E94940832CF8091660281329E
:101CE00009F02DCF80916A0290916B02892B29F522
:101CF0008091E800877F8093E8000E94940880919B
:101D00006802809311010E94D30C809169028F9325
:101D1000809168028F9380916B028F9380916A0209
:101D20008F9386E192E09F938F930E94C0050F905E
:101D30000F900F900F900F900F9080916A029091EA
:101D40006B02019709F0FBCE8091E800877F8093BA
:101D5000E8000E94940880916802809310010E941C
:101D6000D30CEDCE80916602813209F0E8CE8091ED
:101D7000E800877F8093E8000E94940890916802B1
:101D800080916902809323038F939F9380916B02CC
:101D90008F9380916A028F938BE092E01FCF8091A6
:101DA0006602813A09F0CBCE8091E800877F80936C
:101DB000E8008091E80080FFFCCF809123038093AE
:101DC000F1008091E8008E778093E8000E949408EB
:101DD00087E092E00E942705B2CE803889F08238F1
:101DE00049F580916A028F70853020F58093E90073
:101DF0008091EB0085FB882780F91092E90006C0EE
:101E00008091630290916402911182609091E80048
:101E1000977F9093E8008093F1001092F1008091F9
:101E2000E8008E7731C0282F2D7F21F48823F1F030
:101E3000823079F18091E80083FF0AC08091E80048
:101E4000877F8093E8008091EB0080628093EB00B5
:101E50001F701093E900AA960FB6F894DEBF0FBE6C
:101E6000CDBFDF91CF911F910F91089580916802AE
:101E7000813001F7933009F080E080936402109282
:101E8000E9008091E800877F8093E8000E94940831
:101E9000D1CF809168028111F2CF80916A028F7058
:101EA0002FEF280F243030F68093E9002091EB00CB
:101EB00020FFE5CF933031F48091EB008062809376
:101EC000EB00DDCF9091EB0090619093EB0021E06F
:101ED00030E001C0220F8A95EAF72093EA001092C1
:101EE000EA008091EB008860EACF8111A3CF0091D6
:101EF00068020F778091E3008078802B8093E30065
:101F00008091E800877F8093E8000E949408809188
:101F1000E80080FFFCCF8091E30080688093E300BD
:101F200083E0011101C082E080936E0283CF80586C
:101F3000823008F07FCF20916802309169022C3DF9
:101F400083E03807A1F583E08A838AE289834FB76B
:101F5000F894DE01139620E03EE051E2E32FF0E03A
:101F600050935700E49120FF03C0E295EF703F5F6C
:101F7000EF708E2F90E0EA30C0F0C7968D939D935E
:101F80002F5F243159F74FBF8091E800877F8093FE
:101F9000E8006AE270E0CE0101960E940908809193
:101FA000E8008B778093E80045CFC096E7CF80911B
:101FB0006A0290916B02432F55274330510509F473
:101FC0004FC078F54130510509F445C084E590E0F3
:101FD000E6E3F2E04230510509F02CCF2091E80011
:101FE000277F2093E80020916C0230916D028217C8
:101FF000930708F49C0140E02115310509F063C006
:10200000411161C08091E80082FDC9CF80916E02CC
:10201000882329F2853019F28091E80083FFF2CFFE
:10202000BECF4132510509F43FC04232510509F09B
:1020300001CF8330910508F0FDCEFC01EE0FFF1FAC
:10204000E45EFE4F0190F081E02D875E9E4FDC0143
:102050008C9190E01DC082E190E0EAE8F2E0BECF12
:10206000332721303105C1F060F02230310509F00D
:10207000E1CEECE9F2E0E4918E2F90E0ECE9F2E0C1
:1020800007C0ECEEF2E0E4918E2F90E0ECEEF2E08F
:10209000009709F4CFCEA2CFECEDF2E0E4918E2FC1
:1020A00090E0ECEDF2E0F4CF8330910508F0C2CE81
:1020B000880F991FFC01EE5DFE4F0190F081E02D2D
:1020C00089E090E08BCF80916E02882309F467CF7E
:1020D000853009F464CF8091E80083FD60CF809162
:1020E000E80082FD8FCF8091E80080FF85CF80914E
:1020F000F20090E02115310519F08830910550F07B
:1021000041E0089709F040E08091E8008E778093E5
:10211000E80072CF44914093F1003196215031098B
:102120000196E8CF803809F085CE8091E800877F5E
:102130008093E800809165028093F10070CE811158
:1021400079CE00916802023008F074CE8091E800E8
:10215000877F8093E800009365020E949408002323
:10216000B9F084E080936E0280EF92E00E94270530
:1021700042E061EC81E00E94B30842E061EC82E061
:102180000E94B30846E261EC83E00E94B30852CE9D
:102190008091E30087FDE5CF81E0E4CFEF92FF92ED
:1021A0000F931F93CF937C018B010E946508C82F6A
:1021B000811119C08091E80085FD0DC08091E80073
:1021C0008E778093E8000E94690D0E94650888233D
:1021D00089F3C82F08C0F70181917F018093F10036
:1021E0000150110939F78C2FCF911F910F91FF905A
:1021F000EF9008958732D8F58E3108F0FCC08E300C
:1022000009F48FC078F4873009F470C08B3009F47A
:1022100056C0863009F458C08BE495E00E9427052B
:1022200080E00895863109F4A6C078F48031A1F7E2
:1022300090912503892F877F93FF886080932503E2
:1022400083FF7FC085EE96E063C0893109F47CC0CE
:102250008B3111F790912503892F8D7F91FF82603B
:102260008093250381FF5AC08EE197E051C08833E7
:1022700031F150F4893221F0853311F0873261F663
:1022800080E00E94F70C40C08334D1F320F48A33FD
:1022900018F28953F6CF883409F0BECF0E94D30CD0
:1022A00084E497E00E9427052FEF83ED90E321500F
:1022B00080409040E1F700C000000E94EA0781E9F9
:1022C00094E00E94270520C080912503817F8E7FA6
:1022D0008093250384E295E00E94270585E597E039
:1022E0000E94270581E080932403089580912503AF
:1022F00080FF0CC087E397E00E94270580912503AB
:10230000817F8E7F8093250381E008958BE297E0A3
:102310000E942705809125038160F4CF80E197E03A
:10232000D0CF90912503892F8B7F92FF846080937B
:10233000250382FF03C081E097E0EACF81EF96E0BA
:10234000C0CF88ED96E0BDCF89EC96E00E942705CE
:102350008AE996E00E9427058DE496E00E94270511
:1023600087E296E00E94270582EE95E00E9427050D
:1023700086EB95E0A6CF88EA95E00E9427050E94AB
:10238000C7071F928F938EE895E09F938F930E94CB
:10239000C005809111011F928F9387E795E09F936D
:1023A0008F930E94C005809123031F928F9384E630
:1023B00095E09F938F930E94C0052FB7F89480916A
:1023C0001F0390912003A0912103B09122032FBFFE
:1023D000BF93AF939F938F938DE495E09F938F93DB
:1023E0000E94C0058DB79EB742960FB6F8949EBF67
:1023F0000FBE8DBF89CF8D5144CFCF93882309F471
:10240000B1C09CEF980F913A08F058C1C82F809145
:102410002403813071F1F8F0823009F45BC010922E
:102420002403A6E3B2E0EFEF80E09D91C91781F0AD
:10243000EF3F19F4911101C0E82F8F5F8630A9F7A3
:10244000EF3F31F00E2E000CFF0BEC5CFD4FC28312
:10245000CF910C94720C80913402823221F080343E
:1024600011F08038F1F68C2F0E94FA1081117AC099
:10247000D8CF809134028232B1F38034A1F3803816
:1024800091F3C431C9F048F4CB3059F0C031C1F0F8
:1024900082E193E00E94270511C0C93269F0C83378
:1024A000B9F784E295E00E94270588E193E00E9455
:1024B000270581E08170DACF1092240380E0FACF03
:1024C0000E94C00B84E193E00E94270582E0809384
:1024D0002403EFCFC432C8F4CE3108F0BEC0CB30F5
:1024E000E1F040F4C73009F4CFC081EC93E0CF9124
:1024F0000C942705C331C1F1C431B9F7809173023F
:10250000882349F1109273020AC0CB3409F4BAC08F
:10251000C0F4C93299F3C83341F70E94C00B8091CF
:102520007302882309F4C7C01F928F938BEB93E04B
:102530009F938F930E94C0050F900F900F900F9064
:1025400011C0C13509F498C0C23509F48FC0CE342A
:1025500061F66AE092C080ED93E00E94270581E079
:1025600080932403CF9108958AEA93E00E9427057F
:1025700088E993E00E942705809117011F928F93AD
:1025800085E993E09F938F930E94C00583E993E0D0
:102590000E94270581E893E00E942705809116019B
:1025A0001F928F938EE793E09F938F930E94C005B5
:1025B0008CE793E00E9427058DE693E00E942705B3
:1025C000809115011F928F938AE693E09F938F93DA
:1025D0000E94C00588E693E00E94270587E593E006
:1025E0000E942705809114011F928F9384E593E048
:1025F0009F938F930E94C00582E593E00E94270578
:102600008DE393E00E942705809113011F928F9321
:102610008AE393E09F938F930E94C00588E393E041
:102620000E94270581E293E00E9427058091120114
:102630001F928F938EE193E09F938F930E94C0052A
:102640008CE193E00E9427058DB79EB748960FB6A0
:10265000F8949EBF0FBE8DBF62CFCE51EC2FF0E03D
:10266000E85DFE4F80818093730259CF61E08091D5
:1026700073020E946E0A53CF61E0809173020E9440
:10268000EF094DCF6AE0F3CF8EE18093170182E32B
:10269000809316018AE08093150184E180931401F0
:1026A00088E08093130188E28093120183EC93E029
:1026B0000E94270534CF88EB93E019CF90E2980F62
:1026C000983068F4877021E030E001C0220F8A95CD
:1026D000EAF780911203822B80931203B9CE9BE517
:1026E000980F933078F4853A39F0863A41F083E8D0
:1026F00090E0CF910C943E0B81E890E0FACF82E815
:1027000090E0F7CF98E5980F973108F02BCF883AF3
:1027100009F447C0893A09F447C08A3A09F447C026
:102720008B3A09F447C08C3A09F447C08D3A09F452
:1027300047C08E3A09F447C08F3A09F447C0813B3D
:1027400009F447C0803B09F447C0823B09F447C005
:10275000833B09F447C0843B09F447C0853B09F437
:1027600047C0863B09F447C0873B09F447C0883B14
:1027700009F447C0893B09F447C08A3B09F447C0C4
:102780008B3B09F447C08C3B09F447C08D3B09F4EF
:1027900047C08E3B09F447C090E080E0CF910C9495
:1027A000120B82EE90E0FACF89EE90E0F7CF8AEE3E
:1027B00090E0F4CF85EB90E0F1CF86EB90E0EECFA8
:1027C00083EB90E0EBCF84EB90E0E8CF87EB90E0F9
:1027D000E5CF8CEC90E0E2CF8DEC90E0DFCF83E8AA
:1027E00091E0DCCF8AE891E0D9CF82E991E0D6CFC1
:1027F00084E991E0D3CF81E292E0D0CF83E292E00E
:10280000CDCF84E292E0CACF85E292E0C7CF86E2E4
:1028100092E0C4CF87E292E0C1CF8AE292E0BECFDD
:102820008FE690E0BBCF80E790E0B8CFCF92DF9209
:10283000EF92FF920F931F93CF93DF9300D000D0BE
:102840001F92CDB7DEB76C0185E0F601DE0111966F
:1028500001900D928A95E1F7F60140815181238123
:10286000348191E02115310531F05F3F19F491E099
:102870004F3F09F090E090FD99C0F6010281F5808C
:10288000F2949FE0F92249835A830B83722F3D8390
:102890002C83602F8D810E948406182FE92FE295EA
:1028A000EF70EF3008F082C0F0E0E75AFB4E0C9476
:1028B000262268146814A614A6141C154E15D614E6
:1028C000D6144016D61416171617D614D614D217C7
:1028D000F92FFF70FF2E907F19F0F29480EFF8220D
:1028E0000023C9F0FF2039F080911103F82AF092FB
:1028F00011030E94720C812F0F900F900F900F9078
:102900000F90DF91CF911F910F91FF90EF90DF908B
:10291000CF900C94FD11812F0E94300DFF2009F4FF
:1029200045C0F09480911103F822F09211030F90AA
:102930000F900F900F900F90DF91CF911F910F91FB
:10294000FF90EF90DF90CF900C94720C892F8F70D6
:10295000907F903211F08295807F112379F01130B1
:1029600009F449C0002309F455C0FF2059F0F601CD
:10297000958190FF69C29F70958304C0002321F167
:10298000F1100FC00F900F900F900F900F90DF91EC
:10299000CF911F910F91FF90EF90DF90CF900C940B
:1029A000260D21E0F212EECF809310030F900F90CE
:1029B0000F900F900F90DF91CF911F910F91FF908B
:1029C000EF90DF90CF900895F11011C01092100396
:1029D0000F900F900F900F900F90DF91CF911F915C
:1029E0000F91FF90EF90DF90CF900C941B0D91E032
:1029F000F912ECCFDBCF002349F0E5E0EF15B0F2A0
:102A000090911203982309F4BDCFE2CFF4E0FF15B3
:102A100068F2DECFFF20E1F2812F0F900F900F9030
:102A20000F900F90DF91CF911F910F91FF90EF903A
:102A3000DF90CF900C94300D892F8695869583700A
:102A4000C1F0813009F0B2CF812F9370011102C023
:102A500090E080E00F900F900F900F900F90DF911B
:102A6000CF911F910F91FF90EF90DF90CF900C943A
:102A7000120B812F9370011102C090E080E00F9043
:102A80000F900F900F900F90DF91CF911F910F91AA
:102A9000FF90EF90DF90CF900C943E0B002309F451
:102AA00071C0803FA1F40E940406819580931C03AD
:102AB0000F900F900F900F900F90DF91CF911F917B
:102AC0000F91FF90EF90DF90CF900C94D70B813F48
:102AD00019F40E940406EACF823F31F40E940406F2
:102AE000819580931B03E4CF833F19F40E94040671
:102AF000F8CF893F29F40E94C90580931D03D8CFE0
:102B00008A3F21F40E94C9058195F7CF8B3F31F4AC
:102B10000E94C905819580931E03CACF8C3F19F48A
:102B20000E94C905F8CF80911A038160143FA1F07B
:102B300080911A038260153F79F080911A038460B6
:102B4000163F51F080911A038860173F29F0183F13
:102B500031F480911A03806180931A03A9CF809188
:102B6000140381601D3F59F08091140382601E3F61
:102B700031F01F3F09F09CCF809114038460809353
:102B8000140396CF803FC1F480911C0387FD1092FF
:102B90001C0380911B0381118BCF80911C03811139
:102BA00087CF80911D03811183CF80911E038111F6
:102BB0007FCF109215037CCF813F29F480911C03B5
:102BC00018162CF3E6CF80911B03123F29F487FFE0
:102BD000E0CF10921B03DDCF133F19F41816CCF38E
:102BE000D8CF193F39F480911D03181694F610922E
:102BF0001D03CFCF1A3F29F480911D0387FFC9CF52
:102C0000F6CF1B3F39F480911E0387FFC2CF10928D
:102C10001E03BFCF1C3F29F480911E031816BCF37E
:102C2000B8CF80911A038E7F143FA1F080911A03D0
:102C30008D7F153F79F080911A038B7F163F51F0FD
:102C400080911A03877F173F29F0183F31F4809154
:102C50001A038F7E80931A039CCF809114038E7F7A
:102C60001D3F59F0809114038D7F1E3F31F01F3FAF
:102C700009F08FCF809114038B7F8093140389CF49
:102C8000892F837009F064C0011190CE812F829545
:102C900086958770880F880F412F4F70C42ED12CD6
:102CA000F12CE12C082E04C0CC0CDD1CEE1CFF1C0A
:102CB0000A94D2F740E050E0BA0114FF11C00FE0CF
:102CC00010E020E030E004C0000F111F221F331F6E
:102CD0008A95D2F7B901A8014095509560957095F5
:102CE0000091260310912703209128033091290396
:102CF0009695969593709230E9F028F5913089F089
:102D00004C295D296E297F29402351236223732397
:102D1000409326035093270360932803709329035D
:102D200045CEC02AD12AE22AF32A4C295D296E29F0
:102D30007F29EECF4C295D296E297F294027512715
:102D400062277327E5CF4023512362237323EDCFFE
:102D50008695002311F0892F8170882309F426CEEF
:102D6000812F829586958770880F880F412F4F702D
:102D7000C42ED12CF12CE12C082E04C0CC0CDD1C6F
:102D8000EE1CFF1C0A94D2F740E050E0BA0114FF99
:102D900011C00FE010E020E030E004C0000F111F70
:102DA000221F331F8A95D2F7B901A801409550958B
:102DB000609570950091AC021091AD022091AE0229
:102DC0003091AF029695969593709230E9F028F580
:102DD000913089F04C295D296E297F2940235123A8
:102DE000622373234093AC025093AD026093AE0212
:102DF0007093AF02DBCD0C291D292E293F29402BD2
:102E0000512B622B732BEECF4C295D296E297F2924
:102E10004027512762277327E5CF402351236223A0
:102E200073234C295D296E297F29DCCF803F09F46B
:102E30004EC0D0F480E4810F803270F1002309F499
:102E4000ACC0FF2009F4A6C0812F0E94FD111933E8
:102E500009F099C0FFEF21EE84E0F150204080405E
:102E6000E1F700C00000A2CD823F09F470C008F471
:102E70005BC0833F19F7002309F47CC0292F2F7111
:102E800081E090E0A0E0B0E004C0880F991FAA1F85
:102E9000BB1F2A95D2F73AC0E12FE071FE2E892F91
:102EA0008F71002351F00E945107812F8295807FFE
:102EB000F11068CD812F8F7065CD0E942D07812F75
:102EC0008295807FF11084CD812F8F7081CD00237A
:102ED00031F1F4E0FF1508F469CD292F2F7181E05D
:102EE00090E0A0E0B0E004C0880F991FAA1FBB1FAC
:102EF0002A95D2F74091AC025091AD026091AE029A
:102F00007091AF0284279527A627B7278093AC023C
:102F10009093AD02A093AE02B093AF0247CD25E0EF
:102F20002F1508F443CDD9CF892F8F71002399F045
:102F30000F900F900F900F900F90DF91CF911F91F6
:102F40000F91FF90EF90DF90CF900C945107892F55
:102F50008F71002369F30F900F900F900F900F90D7
:102F6000DF91CF911F910F91FF90EF90DF90CF9065
:102F70000C942D071092AC021092AD021092AE028A
:102F80001092AF0213CD133509F464CF173409F052
:102F90000DCD60CF892F8F71CBCFF1103DCD892F13
:102FA0008F71D9CF811102CD002309F4FFCC0E948B
:102FB000D30C8FEF90E7E2E081509040E040E1F7E2
:102FC00000C000000E94EA071F93CF93DF93809117
:102FD0007902807FB1F480917602882391F020916C
:102FE000AB0210917A02C0917402D0917502A09147
:102FF0007702B091780241E0CF3F09F040E0121330
:1030000004C0DF91CF911F91089581E0109721F0C6
:10301000842FDF3F09F080E030E080FD33C0C9013C
:1030200066E070E00E940122FC01E558FD4F8181BD
:103030008D1328C080818C1325C08281811122C00C
:10304000838194818A1B9B0B883C9105D8F48091E5
:1030500079028F70806180937902C90166E070E027
:103060000E940122FC01E058FD4F90819F70906109
:10307000908384E792E00E941614DF91CF911F9114
:103080000C9471072F5F3F4F2770B9CF9F92AF927B
:10309000BF92CF92DF92EF92FF920F931F93CF9345
:1030A000DF93CDB7DEB761970FB6F894DEBF0FBEE2
:1030B000CDBF8C0185E0F801DE011D9601900D92D7
:1030C0008A95E1F7F80140812181F280C380D480A4
:1030D000909174023091750260917702709178023C
:1030E00081E06115710531F03F3F19F481E09F3FA8
:1030F00009F080E0F82FF1709F2E80FD4EC184E72B
:10310000A82E82E0B82EE0907602F601E61BF70BBF
:10311000EE2009F404C180917902582F507FE83CD9
:10312000F10508F0BDC0511183C0EF2C321322C04D
:10313000941320C0F1101EC08F70806180937902BB
:10314000C5010E94161480917902F80185838E2DA5
:1031500061960FB6F894DEBF0FBECDBFDF91CF9161
:103160001F910F91FF90EF90DF90CF90BF90AF90A5
:103170009F90089581E0C114D10431F02F3F19F4DC
:1031800081E04F3F09F080E080FD14C081E08F2591
:10319000F82FF170BF2EE091AB0230917A0280FDE2
:1031A00022C0FF20A1F28091790281608093790290
:1031B000E12CCDCF80E0ECCFF0E0CF0166E070E015
:1031C0000E940122DC01A558BD4F11968C911197E8
:1031D000281307C08C91481304C012968C918F114C
:1031E000E0CF3196E770E313E7CF7C2DD98AC88A08
:1031F000522F6F2D89890E948406292F22952F70C6
:10320000223050F0243078F49F7051F0F80195810D
:10321000907F31F4E92C9BCF9F7011F08823D1F37C
:10322000805E8830B8F3C8010E9416149B2CF2CF40
:10323000321306C0941304C0F801FF2009F48AC0B9
:103240004D872E87FF867C2DD98AC88A522F6F2DF5
:1032500089890E947B07882309F4AEC0FF2009F406
:10326000ABC080917902803270F02091740230916D
:10327000750238872F831986DB86CA868C87CE0134
:1032800007960E94161486E0F801A4E7B2E00190C8
:103290000D928A95E1F70E94E417EE24E39457CF4C
:1032A00051110AC084E792E00E94161486E0F501ED
:1032B00011928A95E9F77CCF32130FC094130DC099
:1032C000F1100BC0F8018583C8010E94161486E036
:1032D000F50111928A95E9F73ACF4D872E87FF863F
:1032E0007C2DD98AC88A522F6F2D89890E947B072D
:1032F000882309F461C0FF2009F45EC0809179023F
:10330000803208F220917402309175023A83298349
:103310001B82DD82CC828E83CE010196B2CFE83C47
:10332000F105A8F6EF2CFF2009F446C032131FC0A8
:1033300094131DC08091790280FD10C0982F907F5A
:1033400069F0F8018583903F31F0982F907F905F6E
:103350008F70892B8583C8010E94161486E0F801BE
:10336000A4E7B2E001900D928A95E1F7F0CE4D8787
:103370002E87FF867C2DD98AC88A522F6F2D898986
:103380000E947B0781117FCF8091790281608093B9
:103390007902C8010E941614DACEFF2069F04D8729
:1033A0002E87FF867C2DD98AC88A522F6F2D898956
:1033B0000E947B07811167CFC8010E9416146DCF50
:1033C000CF93DF93CDB7DEB767970FB6F894DEBF24
:1033D0000FBECDBF4B8B5C8B6D8B7E8B8F8B1A8A18
:1033E000198A85E0FE017396DE011D9601900D920B
:1033F0008A95E1F786E0FE013D96DE011796019081
:103400000D928A95E1F7CE0107960E944618811128
:1034100038C086E0FE013796DE01119601900D92CC
:103420008A95E1F79F8188852A853B85232B39F092
:103430008F3F19F481E09F3F19F080E001C081E0E7
:1034400080FD1FC080917A0290E09C012F5F3F4F6A
:10345000277033274091AB024217130661F166E0F3
:1034600070E00E940122DC01A558BD4F96E0FE01EC
:10347000319601900D929A95E1F720937A020E947D
:1034800071078091AB0290917A02891709F190E05F
:1034900066E070E00E94012285589D4F0E94461808
:1034A0008823B1F08091AB0290E001968770992754
:1034B0008093AB02E6CF0E94D30C10927A02109256
:1034C000AB0286E0E4E7F2E0DF011D928A95E9F7BE
:1034D00067960FB6F894DEBF0FBECDBFDF91CF91D8
:1034E0000895CF93DF9300D01F92CDB7DEB7209120
:1034F0006E02243021F523E029839B838A8382E0B6
:103500008093E9008FEF9091E800815095FD06C00F
:1035100095ED9A95F1F700008111F5CF8091E800C3
:1035200085FF0DC050E040E063E070E0CE01019601
:103530000E94CE108091E8008E778093E8000F9073
:103540000F900F90DF91CF910895CF93DF9300D02C
:103550001F92CDB7DEB720916E02243061F519823B
:103560001A821B8222E029838138910520F080583D
:1035700091099B838A8382E08093E9008FEF909189
:10358000E800815095FD06C095ED9A95F1F7000091
:103590008111F5CF8091E80085FF0DC050E040E03B
:1035A00063E070E0CE0101960E94CE108091E800A9
:1035B0008E778093E8000F900F900F90DF91CF915E
:1035C000089520916E02243049F522E02093E9000D
:1035D0002FEF3091E800215035FD06C035ED3A95CA
:1035E000F1F700002111F5CF2091E80025FF16C06A
:1035F0002091100150E040E063E070E0222339F0B8
:1036000021E02093F10050E040E065E070E00E948E
:10361000CE108091E8008E778093E8000895CF93D4
:10362000DF9320916E02243011F521E02093E90010
:1036300021E8215021F03091E80035FF1BC0209196
:10364000E80025FF14C0EC0150E040E068E070E0C5
:103650000E94CE108091E8008E778093E80088E089
:10366000FE01ABE5B2E001900D928A95E1F7DF91A2
:10367000CF910895EFE3F1E03197F1F700C000003A
:10368000D8CF0E94EC098FEC90E00197F1F700C0D1
:1036900000000E94E9098FE393E00197F1F700C071
:1036A00000000E94EC098FEC90E00197F1F700C058
:1036B00000000E94E9098FED94E00197F1F700C046
:1036C00000000E94EC098FE198E00197F1F700C03B
:1036D00000000C94E9090E94EC098FE094E0019746
:1036E000F1F700C000000E94E9098FEC90E001971B
:1036F000F1F700C000000E94EC098FE692E001970C
:10370000F1F700C000000C94E9098F929F92AF92EC
:10371000BF92CF92DF92EF92FF928FE19EE40197EA
:10372000F1F700C000005E9888E54C9907C00E9440
:10373000960B489906C0789480E094C00E946A0B6A
:10374000F8CF0E946B1BF89480E593EC489B0BC06C
:10375000009719F40E94411BEECFE5E0EA95F1F7DE
:1037600000000197F3CF892BA9F3F5E8FA95F1F75B
:10377000000086E1812C912C540175016401489B65
:1037800002C06894E6F846015701B694A79497944E
:103790008794EFECF0E03197F1F700C00000815022
:1037A00061F7789481149104A104B10429F2811481
:1037B000F6E09F06F0E3AF06B10409F4BDCF5E9AD0
:1037C000E3FA882780F9882309F455C081E50E942F
:1037D000960BE2FA882780F9882309F450C082E525
:1037E0000E94960BE1FA882780F9882309F44BC0E0
:1037F00083E50E94960B84E5E0FE49C00E94960B8B
:10380000D7FA882780F9882309F444C085E50E9407
:10381000960BD6FA882780F9882309F43FC086E5FD
:103820000E94960BD5FA882780F98823D9F187E57D
:103830000E94960BD701C60122E0B695A7959795F1
:1038400087952A95D1F78F7788242FE09222AA2492
:10385000BB24811494E09906A104B10439F50E94B7
:10386000960B81E0FF90EF90DF90CF90BF90AF90EC
:103870009F908F90089581E50E946A0BAACF82E500
:103880000E946A0BAFCF83E50E946A0BB4CF0E94FF
:103890006A0BB6CF85E50E946A0BBBCF86E50E9416
:1038A0006A0BC0CF87E50E946A0BC4CF0E946A0BE7
:1038B000D8CF78941F920F920FB60F9211248F9346
:1038C0009F93AF93BF9380911F0390912003A0918A
:1038D0002103B09122030196A11DB11D80931F0306
:1038E00090932003A0932103B0932203BF91AF9143
:1038F0009F918F910F900FBE0F901F9018951F9260
:103900000F920FB60F9211248F939F93AF93BF9393
:1039100080911303811113C080911F0390912003A4
:10392000A0912103B09122034196A11DB11D809366
:103930001F0390932003A0932103B0932203BF9110
:10394000AF919F918F910F900FBE0F901F90189580
:103950001F920F920FB60F9211242F933F934F9304
:103960005F936F937F938F939F93AF93BF93EF93E7
:10397000FF938091E10082FF09C08091E20082FF05
:1039800005C08091E1008B7F8093E1008091E10090
:1039900080FF23C08091E20080FF1FC08091E20081
:1039A0008E7F8093E2008091E20080618093E2004C
:1039B0008091D80080628093D80019BC85E0809304
:1039C0006E028BEF91E00E94270580915A0280934E
:1039D000590210925A020E94D30C8091E10084FF98
:1039E00031C08091E20084FF2DC084E089BD86E073
:1039F00089BD09B400FEFDCF8091D8008F7D8093F2
:103A0000D8008091E1008F7E8093E1008091E200F8
:103A10008F7E8093E2008091E20081608093E200DB
:103A200080916502882309F448C084E080936E0287
:103A30008FEF91E00E9427050E94D30C80915902DC
:103A400080935A028091E10083FF26C08091E200BA
:103A500083FF22C08091E100877F8093E10082E0B4
:103A600080936E02109265028091E1008E7F8093B8
:103A7000E1008091E2008E7F8093E2008091E2007D
:103A800080618093E20042E060E080E00E94B30841
:103A900083E092E00E942705FF91EF91BF91AF91E3
:103AA0009F918F917F916F915F914F913F912F9156
:103AB0000F900FBE0F901F9018958091E30087FD27
:103AC00002C081E0B3CF83E0B1CFCF93DF93CDB716
:103AD000DEB72C970FB6F894DEBF0FBECDBF84B70C
:103AE000877F84BF0FB6F894A895809160008861A5
:103AF00080936000109260000FBE80E890E00FB6E7
:103B0000F89480936100909361000FBE80E099E08B
:103B1000909333018093320186E091E090931703F4
:103B20008093160382EE91E00E9427050E94D3073E
:103B3000809163008E7F8093630081E080935802C0
:103B40001092E2001092E1008091D8008F7780936C
:103B5000D8008091D80080688093D8008091D800E8
:103B60008F7D8093D80084E089BD86E089BD09B44B
:103B700000FEFDCF10926E02109265021092640258
:103B80001092630242E060E080E00E94B3088091FE
:103B9000E1008E7F8093E1008091E200816080935C
:103BA000E2008091E20088608093E2008091E00072
:103BB0008E7F8093E000789482E084BD93E095BD91
:103BC0009AEF97BD80936E0080912503816080936A
:103BD00025032FEF34E34CE0215030404040E1F723
:103BE00000C000008091250380FF08C080E891E0BC
:103BF0009F938F930E94C0050F900F90569A5E9AE4
:103C000054985C9A0E94E9095098589A0E946B1B3C
:103C10008FE094E00197F1F700C000000E94411B83
:103C2000EFE7F6E03197F1F700C000000E946B1B50
:103C30008FE094E00197F1F700C000000E94411B63
:103C4000EFE7F6E03197F1F700C0000089E492E079
:103C5000BDE3CB2EB2E0DB2EF60111926F018E1781
:103C60009F07D1F78091250380FF08C081E691E08E
:103C70009F938F930E94C0050F900F9080916E02CA
:103C8000843009F062C10E94E808882309F45DC10C
:103C900080ED91E00E94270582EC91E00E942705CB
:103CA000F7EB4F2EF1E05F2EA8E16A2E712C809188
:103CB0006E02853009F44CC10E94851B0AE412E0B3
:103CC000EDE3AE2EE2E0BE2E312CF50121905F0136
:103CD000F8019080921409F468C08091250381FF57
:103CE00040C08AEA91E00E9427052DE332E03C873C
:103CF0002B87F12CE12CEB85FC852191FC87EB8750
:103D0000229530E0C901880F991F880F991F8C7C7C
:103D100035952795359527952373822B90E028E1DB
:103D200031E03F932F939C01220F331F2A7A959500
:103D300087958575822B1F928F93FF92EF928FE963
:103D400091E09F938F930E94C005FFEFEF1AFF0A47
:103D50000FB6F894DEBF0FBECDBF3CE0E316F10412
:103D600051F6E12CFF24F3949224892D8F21C1F088
:103D7000EE823F8291E08F2D822109F490E09887B6
:103D80000E9478068160782F9A8789874E815F81AB
:103D900068858A850E94E019F80180818F258083DB
:103DA000E394FF0CF8E0EF12E0CF33940F5F1F4F66
:103DB0002CE032128ACF3FEF39833A831B820E9474
:103DC00078068160782F9D838C8349815A816B812D
:103DD0008D810E94E01980911803909119032FB7EB
:103DE000F89440911F03509120036091210370913A
:103DF00022032FBFFA01E81BF90B209115038091D4
:103E0000160190E0211107C08091170190E06AE04F
:103E100070E00E940122E817F90780F080911B03EF
:103E2000F0901C0310911D0300911E038111C6C068
:103E3000F110AAC11111A8C10111A6C10E94C707A2
:103E400090914902891709F44BC00E94C7078093DB
:103E50004902909125039570953051F41F928F93EC
:103E60005F924F920E94C0050F900F900F900F909D
:103E70008091490281FF10C1F8940E94EC098FE4FF
:103E800097E00197F1F700C000000E94E909EFE612
:103E9000F2E03197F1F700C000000E94EC098FECCE
:103EA00090E00197F1F700C000000E94E909EFECF3
:103EB000F0E03197F1F700C000000E94E9098FECB3
:103EC00090E00197F1F700C000000E94EC09EFEAD2
:103ED000F5E03197F1F700C000000E94E9097894FD
:103EE0002091E4003091E5008091560290915702B4
:103EF0002817390739F18091E4009091E5009093FB
:103F00005702809356020E94E8088823D9F08091D6
:103F10006E028430B9F48091E9008F709091EC00CA
:103F200090FFDEC090E8892B93E09093E900909198
:103F3000EB0090FF04C09091EE0097FDEFC08F70F2
:103F40008093E9000E94690DB2CE0E94690D96CE61
:103F500080916E02843011F11092130380E40FB649
:103F6000F894A895609260000FBE8093600083B7BC
:103F7000817F846083BF83B7816083BF7894889595
:103F800083B78E7F83BF0FB6F894A89580916000A9
:103F9000886180936000109260000FBE809164027F
:103FA000882309F484CE0E94851BEDE3F2E0819121
:103FB0008111D4C0CE16DF06D1F779CE2F3F19F08C
:103FC0002F5F20931503181624F40E940406809393
:103FD0001B0380911B0387FF05C00E940406819587
:103FE00080931B031F1424F40E94040680931C0377
:103FF00080911C0387FF05C00E9404068195809371
:104000001C0360911B03662331F1F0901C03FF2019
:1040100011F1062E000C770B880B990B0E940021E2
:1040200023E333E343E35FE30E9464210E94C8205B
:1040300060931B036F2DFF0C770B880B990B0E946D
:10404000002123E333E343E35FE30E9464210E9402
:10405000C82060931C03111624F40E94C9058093A4
:104060001D0380911D0387FF05C00E94C90581952E
:1040700080931D03101624F40E94C90580931E032B
:1040800080911E0387FF05C00E94C905819580931A
:104090001E030E94D70BD2CEF8940E94EC098FE445
:1040A00097E00197F1F700C000000E94E909EFE6F0
:1040B000F2E03197F1F700C000000E94EC098FECAC
:1040C00090E00197F1F700C000000E94EC09EFECCE
:1040D000F0E03197F1F700C000000E94EC09EFCE4C
:1040E00090E021CFE0910101F0910201E90FF11D73
:1040F00020819F5F309105019323909304012093C9
:10410000F1009091E80095FD09C09091E80090FFC2
:1041100005C09091E8009E779093E800909104018B
:1041200020910301291721F02091E80025FDDACF25
:104130009091F200992309F402CF9091E80090FF4A
:10414000FECE9091E80095FD06C09091E8009E7724
:104150009093E800F4CE1092F100F3CF84E089BD93
:1041600086E089BD09B400FEFDCF8091D8008F7D27
:104170008093D8008091E00082608093E00080917D
:10418000E00081FDFCCF93CD2F3F09F019CF2ACF5E
:104190000E94CF206894B1110C945E2108950E9472
:1041A000432188F09F5798F0B92F9927B751B0F065
:1041B000E1F0660F771F881F991F1AF0BA95C9F7AB
:1041C00014C0B13091F00E945D21B1E008950C94CB
:1041D0005D21672F782F8827B85F39F0B93FCCF37E
:1041E000869577956795B395D9F73EF49095809528
:1041F000709561957F4F8F4F9F4F0895E89409C048
:1042000097FB3EF490958095709561957F4F8F4F09
:104210009F4F9923A9F0F92F96E9BB279395F6951F
:10422000879577956795B795F111F8CFFAF4BB0F9D
:1042300011F460FF1BC06F5F7F4F8F4F9F4F16C001
:10424000882311F096E911C0772321F09EE8872F8B
:10425000762F05C0662371F096E8862F70E060E047
:104260002AF09A95660F771F881FDAF7880F9695C0
:10427000879597F9089557FD9058440F551F59F0A9
:104280005F3F71F04795880F97FB991F61F09F3F43
:1042900079F087950895121613061406551FF2CF6C
:1042A0004695F1DF08C0161617061806991FF1CFBC
:1042B00086957105610508940895E894BB276627E3
:1042C0007727CB0197F908950E9476210C94F0216D
:1042D0000E94E22138F00E94E92120F0952311F09C
:1042E0000C94D9210C94DF210C945E210E943B2177
:1042F00078F39923C9F35523B9F3950F50E0551F6F
:10430000AA27EE27FF27BB2700240894679520F4EF
:10431000E20FF31FB41F0A1E220F331F441FAA1FF0
:104320006695A9F7779530F4F30FB41F0A1E121E95
:1043300008F46395330F441FAA1F221F769599F73F
:10434000879520F4B40F0A1E121E631F440FAA1F84
:10435000221F331F8695A9F7862F712D602D1124FA
:104360009F5750409AF0F1F088234AF0EE0FFF1F5C
:10437000BB1F661F771F881F91505040A9F79E3FB3
:10438000510580F00C94D9210C945E215F3FE4F339
:10439000983ED4F3869577956795B795F795E79509
:1043A0009F5FC1F7FE2B880F911D9695879597F912
:1043B000089597F99F6780E870E060E008959FEFA7
:1043C00080EC089500240A941616170618060906AC
:1043D000089500240A94121613061406050608957B
:1043E000092E0394000C11F4882352F0BB0F40F403
:1043F000BF2B11F460FF04C06F5F7F4F8F4F9F4F43
:1044000008950024552704C0080E591F880F991FCE
:10441000009729F076956795B8F37105B9F7802D67
:10442000952F089597FB072E16F4009407D077FD7B
:1044300009D00E942C2207FC05D03EF4909581956E
:104440009F4F0895709561957F4F0895EE0FFF1F60
:104450000590F491E02D0994AA1BBB1B51E107C004
:10446000AA1FBB1FA617B70710F0A61BB70B881F04
:10447000991F5A95A9F780959095BC01CD01089593
:04448000F894FFCFDE
:104484000534010000FFE5080F1BE11AA51A711A93
:1044940001012808140A321E00407F2215019600EB
:1044A4007400480261027A02010203040506070847
:0244B4000900FD
:106800000000000000000000040005000600070072
:10681000080009000A000B000C000D000E000F001C
:1068200010001100120013001400150016001700CC
:10683000180019001A001B001C001D001E001F007C
:10684000200021002200230024002500260027002C
:10685000280000002A002B002C002D002E002F0005
:1068600030003100000033003400290036003700CA
:106870003800E00000000000000000000000000000
:106880000000000000000000000000000000000008
:106890000000E944E2444B00EA4400004E004F008F
:1068A0005000510052003500310054005500560090
:1068B000580059005A005B005C005D005E005F00FC
:1068C00060006100620063000000F1A15700000059
:1068D00000000000000000000000000000000000B8
:1068E00000000000000000000000000000000000A8
:1068F000E200E1000000E300E600E5000000000027
:106900000100010001000100EA4401000601E24427
:106910000100010001005500460054004A004B00F0
:10692000560057004700480031000100E9440100CB
:106930000100190101001B0101001D013A003B008B
:106940003C003D003E003F0040004100420043004B
:10695000010001004C0039000100440045005200D4
:1069600049000100010050004F0035004D004E006D
:1069700051000100010001000100010001000100BF
:1069800001000100010001000100010001000100FF
:1069900001000100010001000100010001004D00A3
:1069A0004A004E004B0053000100010001000100AD
:1069B00001000100010001000100010001000100CF
:1069C00001000100010001000100010001000100BF
:1069D00001000100010001000100010001000100AF
:1069E000010001000100010001000100010001009F
:1069F000010001000100010001000100010001008F
:00000001FF
